:100000000528FF3FFF3FFF3FD82E03138316013023
:100010008500E1308600003087000130880007301D
:100020008900831230309000831602309F008312C3
:1000300081309F0083168F308100831210308B0037
:100040006400860187018801C001C101C201C301AA
:10005000C401C501C601C701C80188148817C82694
:100060000611861001308700861500008611C8260B
:10007000071002308700861500000711C826861079
:1000800006308700861500008611C82686100C30C1
:100090008700861500008611C82686101430870058
:1000A000861500008611C826861038308700861510
:1000B00000008611C8268610403087008615000093
:1000C0008611C82686140030870086150000861128
:1000D000C826861400308700861500008611C826C1
:1000E000861400308700861500008611C826861405
:1000F00009308700861500008611C826861409304D
:100100008700861500008611C826861417308700E0
:10011000861500008611C8268614103087008615C3
:1001200000008611C826861410308700861500004E
:100130008611C826861410308700861500008611A7
:10014000C826861000308700861500008611C82654
:10015000861048308700861500008611C826861450
:1001600004308700861500008611C82686140430E6
:100170008700861500008611C82686141F30870068
:10018000861500008611C82686140430870086155F
:1001900000008611C82686140430870086150000EA
:1001A0008611C82686140430870086150000861143
:1001B000C826861400308700861500008611C826E0
:1001C00086141F308700861500008611C826861405
:1001D00000308700861500008611C8268610003082
:1001E0008700861500008611C826F628E221B82669
:1001F000A621B826B826B8262422B826B826B826BE
:10020000B826091906296622B826B826A8229C21F4
:100210001B29A6213C243324431CD221091D11296A
:100220001429C319DA211729431ADA211729861A42
:10023000C621B8269C21091C1E2929292B212B21E6
:100240002B212B212B212B212B212B212B212B214E
:1002500009292B2109298E018F01C6010C100811D3
:10026000101464000C18C60A0C180C10C6190815D6
:10027000C619DA21061831298E018F01C6010C102A
:100280000811101447106400061857290C18C60AE4
:10029000061857290C180C1006185729C6190815E6
:1002A00006185729C619DA210618572943290816AE
:1002B0008B108B17091C962160218B1308120800E4
:1002C00008188810471808006821431A0800602998
:1002D000061C47146400BC0ABC18BC1D7229BB0A6A
:1002E000BC014314BB18BB1D7829BA0ABB01C31457
:1002F000BA18BA1D7E29B80ABA014315B818B81D34
:100300008429B70AB801C315B718B71D8A29B60AD8
:10031000B7014316B618B61D0800BC01BB01BA01EF
:10032000B801B701B601C301081508004630C00086
:10033000C00B982964000800B601B701B801BA01E2
:10034000BB01BC01FE30B400C30108001F151F191A
:10035000A729AA299E1BBC290612B42408138812B7
:10036000B82608178816B82608138812B826081762
:100370008816B826881008000817881206121E1B57
:10038000C229080008138816061608000D238815D0
:10039000C8266400861AC929B8266400861ECD299D
:1003A0008811080008150918332409186F23091C3F
:1003B000F123080008150919332409192F23091DF1
:1003C000AF2308004D30A0004530A1005230A200FC
:1003D0004930A3004330A400FE30A5004B30A600F6
:1003E0004130A7005030A8004130A9004330AA0096
:1003F0004930AB005430AC005930AD00FE30AE0097
:10040000FE30AF00FE30B000FE30B100FE30B20072
:100410004D30B3002E30B4004F30B5004C30B60034
:100420004530B7004A30B8004130B9005230BA0008
:100430002C30BB003230BC003030BD003030BE004C
:100440003330BF00F62408003130A0003030A10066
:100450007030A2004630A300FE30A400FD30A5009D
:10046000FE30A6003130A7003030A8006D30A90062
:100470004630AA00FE30AB00FE30AC00FE30AD00CE
:10048000FE30AE00FE30AF000130B0003130B100C0
:100490002530B200FE30B300FE30B400FE30B500AF
:1004A000FE30B600FE30B7004530B8004C30B90021
:1004B0005730BA004530BB004230BC002E30BD0082
:1004C0004330BE005A30BF00F62408005030A00070
:1004D0004F30A1005A30A2004F30A3005230A40088
:1004E000FE30A500FE30A6004E30A7004130A80027
:1004F000FE30A900FE30AA00FE30AB00FE30AC009A
:10050000FE30AD00FE30AE00FE30AF00FE30B00079
:10051000FE30B100FE30B200FE30B300FE30B40059
:10052000FE30B500FE30B600FE30B7005030B800E7
:100530004F30B9004C30BA004130BB005230BC00E3
:100540004930BD005430BE005530BF00F6240800CD
:10055000FF30A000A100A200A300A400A500A600F7
:10056000A700A800A900AA00AB00AC00AD00AE0037
:10057000AF00B000B100B200B300B400B500B600E7
:10058000B700B800B900BA00BB00BC00BD00BE0097
:10059000BF00F62408004B30A0004130A1005030CD
:1005A000A2004130A3004330A4004930A5005430DC
:1005B000A6004130A700FE30A800FE30A900FE30A2
:1005C000AA00FE30AB00FE30AC00FE30AD00FE30C5
:1005D000AE00FE30AF004330B0003D30B100FE3021
:1005E000B200FE30B300FE30B400FE30B500FE3085
:1005F000B600FE30B700FE30B800FE30B900FE3065
:10060000BA00FE30BB00FE30BC00FE30BD00FE3044
:10061000BE004630BF00F62408004B30A000413039
:10062000A1005030A2004130A3004330A400493063
:10063000A5005430A6004130A700FE30A80042308B
:10064000A9005930AA004C30AB004130AC00FE305C
:10065000AD00FE30AE00FE30AF00F62408005A3088
:10066000A0004D30A1004530A2004E30A300543010
:10067000A4004530A500FE30A6005230A7004F3040
:10068000A8005A30A9005330AA004130AB004830CE
:10069000AC00FE30AD00FE30AE007E30AF00433027
:1006A000B000FE30B100FE30B200FE30B3003E308C
:1006B000B400FE30B5003130B6003030B700303015
:1006C000B800FE30B9003030BA003030BB003030F6
:1006D000BC00FE30BD004630BF00F62408005A3092
:1006E000A0004D30A1004530A2004E30A300543090
:1006F000A4004530A500FE30A6005230A7004F30C0
:10070000A8005A30A9005330AA004130AB0048304D
:10071000AC00FE30AD00FE30AE007F30AF004330A5
:10072000B000FE30B100FE30B200FE30B300FE304B
:10073000B400FE30B500FE30B600FE30B700FE302B
:10074000B8003C30B900FE30BA003130BB00303068
:10075000BC00FE30BD004630BF00F62408004B3020
:10076000A0004130A1005030A2004130A30043302E
:10077000A4004930A5005430A6004130A700FE3047
:10078000A8004A30A9004530AA00FE30AB00FE3078
:10079000AC00FE30AD00FE30AE00FE30AF00FE30EB
:1007A000B000FE30B100FE30B200FE30B300503079
:1007B000B4005230B5004930B6004C30B700493073
:1007C000B8005330B900FE30BA005630BB00453097
:1007D000BC004C30BD004B30BE004130BF00F624A1
:1007E00008004B30A0004130A1005030A200413041
:1007F000A3004330A4004930A5005430A600413086
:10080000A700FE30A8004A30A9004530AA00FE30FB
:10081000AB00FE30AC00FE30AD00FE30AE00FE306E
:10082000AF00FE30B000FE30B100FE30B200FE304E
:10083000B300FE30B4005030B5005230B60049303D
:10084000B7004C30B8004930B9005330BA00FE3020
:10085000BB004D30BC004130BD004C30BE004130CB
:10086000BF00F6240800091C7030891C6E30091D79
:100870000030BE00F624080009194A2C3B08BC00D1
:100880003A08BB003808BA003708B8003608B70085
:10089000B601C30C4B30A0004130A1005030A20083
:1008A0004130A3004330A4004930A5005430A600D5
:1008B0004130A700FE30A800FE30A900FE30AA009B
:1008C000FE30AB00FE30AC00FE30AD00FE30AE00BE
:1008D000FE30AF004330B0003D30B100FE30B2001A
:1008E000FE30B300FE30B400FE30B500FE30B9007B
:1008F000FE30BD004630BF003616B6163613B613AE
:100900003716B7163713B7133816B8163813B81387
:100910003A16BA163A13BA133B16BB163B13BB135F
:100920003C16BC163C13BC1343189A2C3B12BB1646
:100930003B13BB17C318A02C3A12BA163A13BA17B6
:100940004319A62C3812B8163813B817C319AC2C93
:100950003712B7163713B717431AB22C3612B6161A
:100960003613B617F62408004E30A0004930A10017
:100970005A30A2004B30A3004530A400FE30A50041
:100980004E30A6004130A7005030A8004130A900E9
:100990004A30AA004530AB004330AC004930AD00CE
:1009A000FE30AE00FE30AF004E30B0004130B1003E
:1009B0005030B2004530B3005430B4004930B50077
:1009C000FE30B600FE30B700FE30B800FE30B90091
:1009D000FE30BA00FE30BB00FE30BC002130BD004E
:1009E0002130BE002130BF00F6240800D226861038
:1009F00080308700861500008611D22686142008D4
:100A00008700861500008611D22686108130870067
:100A1000861500008611D2268614210887008615C7
:100A200000008611D22686108230870086150000CD
:100A30008611D226861422088700861500008611AA
:100A4000D226861083308700861500008611D226B4
:100A5000861423088700861500008611D22686108A
:100A600084308700861500008611D226861424085B
:100A70008700861500008611D226861085308700F3
:100A8000861500008611D226861425088700861553
:100A900000008611D2268610863087008615000059
:100AA0008611D22686142608870086150000861136
:100AB000D226861087308700861500008611D22640
:100AC000861427088700861500008611D226861016
:100AD00088308700861500008611D22686142808E3
:100AE0008700861500008611D2268610893087007F
:100AF000861500008611D2268614290887008615DF
:100B000000008611D22686108A30870086150000E4
:100B10008611D22686142A088700861500008611C1
:100B2000D22686108B308700861500008611D226CB
:100B300086142B088700861500008611D2268610A1
:100B40008C308700861500008611D22686142C086A
:100B50008700861500008611D22686108D3087000A
:100B6000861500008611D22686142D08870086156A
:100B700000008611D22686108E3087008615000070
:100B80008611D22686142E0887008615000086114D
:100B9000D22686108F308700861500008611D22657
:100BA00086142F088700861500008611D22686102D
:100BB000C0308700861500008611D22686143008C2
:100BC0008700861500008611D2268610C130870066
:100BD000861500008611D2268614310887008615F6
:100BE00000008611D2268610C230870086150000CC
:100BF0008611D226861432088700861500008611D9
:100C0000D2268610C3308700861500008611D226B2
:100C1000861433088700861500008611D2268610B8
:100C2000C4308700861500008611D2268614340849
:100C30008700861500008611D2268610C5308700F1
:100C4000861500008611D226861435088700861581
:100C500000008611D2268610C63087008615000057
:100C60008611D22686143608870086150000861164
:100C7000D2268610C7308700861500008611D2263E
:100C8000861437088700861500008611D226861044
:100C9000C8308700861500008611D22686143808D1
:100CA0008700861500008611D2268610C93087007D
:100CB000861500008611D22686143908870086150D
:100CC00000008611D2268610CA30870086150000E3
:100CD0008611D22686143A088700861500008611F0
:100CE000D2268610CB308700861500008611D226CA
:100CF00086143B088700861500008611D2268610D0
:100D0000CC308700861500008611D22686143C0858
:100D10008700861500008611D2268610CD30870008
:100D2000861500008611D22686143D088700861598
:100D300000008611D2268610CE308700861500006E
:100D40008611D22686143E0887008615000086117B
:100D5000D2268610CF308700861500008611D22655
:100D600086143F088700861500008611D2260800E9
:100D70001430C2006430C1006430C0006400081840
:100D80008810C00BC12EC10BBC2EC20BBA2E08009E
:100D90000A30C1006430C000C00BCC2EC10BCA2E7B
:100DA000640008003C30C000C00BD42E6400080072
:100DB0008B1047140900FF3FFF3FFF3FFF3FFF3FFE
:100DC000FF3FFF3FFF3FFF3FFF3FFF3FFF3FFF3F33
:100DD000FF3FFF3FFF3FFF3FFF3FFF3FFF3FFF3F23
:100DE000FF3FFF3FFF3FFF3FFF3FFF3FFF3FFF3F13
:100DF000FF3FFF3FFF3FFF3FFF3FFF3FFF3FFF3F03
:02400E00F93F78
:08400000FF3FFF3FFF3FFF3FC0
:00000001FF
